:100000008328A600360884000930A70003100D20BD
:10001000A60CA70B072803140D288413B31D1C2856
:1000200000083404331D34068000841700083404AB
:10003000031C34068000272800083404031C3406FF
:100040003319340680008417340980052728330DBE
:100050000639A0003020A100A00A302000003D2871
:1000600000308A002008820701349934033439347F
:10007000003460340C34FD34A101FC3EA000A10921
:10008000031C4828FF300000A00703184328A007DE
:100090006400A10F42280800A20001305228A200EB
:1000A00006305228A80023082102031D59282208DF
:1000B0002002043003180130031902302805031D03
:1000C000FF307E28A501A4011030A600210DA40D4B
:1000D000A50D2208A4022308031C230FA502031860
:1000E00078282208A40723080318230FA507031064
:1000F000A00DA10DA60B662820087E2883130313EC
:1001000083126400080007309F00831606118312D3
:1001100006118316061106128312061683160610A0
:1001200085168312B801B9010130BB0064000930A3
:100130003B0203186329061483160610831200007D
:1001400000000000000000000000000000000000AF
:10015000000000000000000000000000000000009F
:10016000000000000000000000000000000000008F
:10017000000000000000000000000000000000007F
:10018000000000000000000000000000000000006F
:10019000000000000000000000000000000000005F
:1001A000000000000000000000000000000000004F
:1001B000000000000000000000000000000000003F
:1001C000000000000000000000000000000000002F
:1001D000000000000000000000000000000000001F
:1001E0000000000000000000000000000610831660
:1001F0000610831200000000000000000000000054
:1002000000000000000000000000000000000000EE
:1002100000000000000000000000000000000000DE
:1002200000000000000000000000000000000000CE
:1002300000000000000000000000000000000000BE
:1002400000000000000000000000000000000000AE
:10025000000000000000000000000000000000009E
:10026000000000000000000000000000000000008E
:10027000000000000000000000000000000000007E
:10028000000000000000000000000000000000006E
:10029000000000000000000000000000000000005E
:1002A000000000000000000000000000000000004E
:1002B000000000000000000000000000000000003E
:1002C0000000BB0F962802303C20B80A0319B90A77
:1002D0003808A0003908A1000130A300F4304F20F5
:1002E000031D7429BA0185296400851A6529380817
:1002F000A0003908A100A30102304C20031D82296F
:10030000BA018529390C380CBA000630B600043021
:10031000B4000630B3003A080120B801B90110302A
:0A0320008606831606128312942845
:02400E00453F2C
:00000001FF
